:020000020000FC
:100000000C943C000C943C000C943C000C943C0080
:100010000C943C000C943C000C943C000C943C0070
:100020000C943C000C943C000C943C000C943C0060
:100030000C943C000C943C000C94FB000C943C0091
:100040000C943C000C943C000C943C000C943C0040
:100050000C943C000C94DD000C943C000C943C008F
:100060000C943C000C943C005472525F4244545235
:100070004D495F56302E3033F894A89500916000BA
:100080000861009360000FE00093600004E00EBF81
:100090000FEF0DBF04B700930001007604BF2224C8
:1000A000B1E0A0E02D92B330E9F706E010E004B92A
:1000B00015B90FE310E007B918B90AE012EE0AB952
:1000C0001BB96BD42DD402E004BD02E005BD0DE7E1
:1000D00007BD02E000936E0003E20093B00002E06F
:1000E0000093B10002E80093B4000CE800937A009A
:1000F00007E600937C0010E00FE01093C50000932A
:10010000C40008E10093C10006E00093C200209201
:100110000401332708E0502E04E0602E0AEF702E11
:10012000AA24BB2444276627552783E001E40093D3
:10013000300102E4009340010AE30093310100938F
:10014000410110E020E013D30F3F69F010E020E000
:10015000A0E6B1E0CAE00BD30D9301E0100F221D21
:10016000CA95C9F71EC004E2009360010AE000933B
:10017000610102E30093620105E00093630100E086
:100180000093640105E2009365010AE000936601B3
:1001900002E30093670105E00093680100E000932B
:1001A00069017894A89501D421D255D2BDD2DCD072
:1001B000AAD125D108D17ED1F5CFCFB6CF920F935A
:1001C00000917C00017049F40091790000930601D0
:1001D00000917C00007F076008C0009179000093C7
:1001E000050100917C00007F066000937C000F9168
:1001F000CF90CFBE1895CFB6CF920F931F9300919B
:100200007A00006400937A00839493945A9419F4CA
:1002100008E0502E01C0A3C0009162010A1519F038
:1002200030F0A39404C020920901A3942A9800916D
:1002300067010B1519F030F0B39404C020920A0145
:10024000B394299800910D01003021F00A95009394
:100250000D0149F000910E010030C1F00A950093A4
:100260000E0159F013C000E81091610111501F7088
:10027000012B00935001716009C000E810916601E4
:1002800011501F70012B0093530172600091010106
:10029000016000930101009101014E9B04C03324D1
:1002A0000093010119C04F9B17C01FEF3116A1F039
:1002B000339412E0311681F40860009301014D99E6
:1002C00006C0009101010B7F0093010105C0009160
:1002D00001010460009301016A9481F405E0602E3D
:1002E000009101011FEF411651F043941AEF41169E
:1002F00031F402600061009301010DC030C04F9BDA
:100300000AC01AE0411630F01AEF411618F40260E4
:1003100000930101442400910B01002319F00A9578
:1003200000930B0100910C01002319F00A95009332
:100330000C017A94A1F408EC702E0091040103954D
:100340000093040100911101002349F00A950093E4
:10035000110129F4009102010B7F009302011F910A
:100360000F91CF90CFBE18950091C00007FF089560
:100370002091C0000091C6002C7131F02091C00086
:100380000091C60083E00895B1E0A7E507FD03C032
:10039000833039F40895093B09F008950C938827B8
:1003A0000895A80FB21D0C938395823009F008952B
:1003B00083E000910201046008600093020103E001
:1003C0000093110108950091020100FF08950E7F2E
:1003D000009302012A9A299A10E020E0A0E6B1E0F9
:1003E000CAE0C5D1102E0D91011509F0B4D101E07C
:1003F000100F221DCA95A9F72A98299808950091EF
:10040000020101FD02C002FF0895E0E8F7E0C3E346
:10041000D1E01DE000E209931A95E9F723961DE06B
:1004200009931A95E9F76D976A3009F466276530E4
:1004300008F0609610E1619FE00DF11D1127059114
:10044000003019F009931395FACF059100930F012D
:100450000591009310010091010105FF08C00F7D77
:1004600000930101A0E6B1E0A60FB21D5C9100E28D
:100470000993052F0BD300911001043608F0F9926F
:100480000A3008F0E992D992603019F0653009F02D
:10049000089500E20993052FE0E2F8E00C5013E024
:1004A000019FE00DF11D05910993059109930491B8
:1004B000088308950091020101FD089502FD089549
:1004C00000910B01B1E0A3E31FEF2DE0093028F00C
:1004D00009501D932A95D1F708951DE21D932A9581
:1004E000E9F700910C01B1E0A3E41FEF2DE0093022
:1004F00028F009501D932A95D1F708951DE21D9308
:100500002A95E9F708950091010101FD29C003FD35
:1005100005C00091020103FD3BC00895077F0093D1
:1005200001010091020101FF08950091010102FF04
:1005300009C000910F01501719F4509110010AC021
:100540005A9508C000911001501719F450910F01ED
:1005500001C05395A0E6B1E0A60FB21D5C930895CB
:100560000D7F00620093010104FD02C063950895B0
:10057000009101010F7E00930101009102011127FA
:100580001260012701FF01600093020166270895B0
:10059000077F0093020100915701045108F10A30CE
:1005A000F8F4602F50915801E0E8F7E010E1619F06
:1005B000E00DF11D0591003009F0FCCF059100938D
:1005C0000F0105910093100100910F01501710F4D5
:1005D000502FC0CF00911001501708F0502FBACF04
:1005E000009102010B7F0093020108950091050123
:1005F000003810F0005803C010E8101B012F00381D
:1006000008F00FE70093070110910B01011710F09C
:1006100000930B0110910901011710F000930901DB
:1006200000910601003810F0005803C010E8101BBC
:10063000012F003808F00FE70093080110910C011A
:10064000011710F000930C0110910A01011710F02E
:1006500000930A010895109162011A1578F500912E
:10066000090110916301011720F40091070101179E
:1006700028F10FE0801609F022C0AA242A9A00E986
:100680001091610111501F70012B009350010091D6
:100690006001009351011091640100910901019FD3
:1006A000112021F4000D003808F401C00FE7009379
:1006B00052010AE000930D01716001C0882410917D
:1006C00067011B1578F500910A0110916801011767
:1006D00020F400910801011728F10FE0901609F0AD
:1006E0000895BB24299A00E91091660111501F70EA
:1006F000012B009353010091650100935401109167
:10070000690100910A01019F112021F4000D0038B8
:1007100008F401C00FE7009355010AE000930E01B1
:10072000726008959924089570FD03C071FD05C09D
:100730000895B1E0A0E57E7F03C0B1E0A3E57D7F31
:1007400013E00091C00005FFFCCF0D910093C6009F
:100750001A95B9F70895F894F999FDCFF89422BD48
:1007600011BD00BDFC98FA9AF99A78940895F99908
:10077000FECFF89422BD11BDF89A00B57894089583
:100780004E6F74653A001860000000000000000021
:100790004368616E6E656C3A000110000000000055
:1007A00052656C656173653A0014FA000000000040
:1007B000476174653A000546000000000000000033
:1007C00056656C6F636974793A0000080000000098
:1007D0004E6F74653A0018600000000000000000D1
:1007E0004368616E6E656C3A000110000000000005
:1007F00052656C656173653A0014FA0000000000F0
:10080000476174653A0005460000000000000000E2
:1008100056656C6F636974793A0000080000000047
:100820004330204323304430204423304530204699
:1008300030204623304730204723304130204123A9
:10084000304230204331204323314431204423318E
:10085000453120463120462331473120472331415D
:10086000312041233142312043322043233244326C
:10087000204423324532204632204623324732205C
:100880004723324132204123324232204333204336
:100890002333443320442333453320463320462337
:1008A000334733204723334133204123334233201E
:1008B00043342043233444342044233445342046F5
:1008C0003420462334473420472334413420412305
:1008D00034423420433520432335443520442335E6
:1008E00045352046352046233547352047233541B9
:1008F00035204123354235204336204323364436C4
:1009000020442336453620463620462336473620B7
:1009100047233641362041233642362043372000D4
:1009200098D097D00CE008B900000000419A000070
:1009300000000000419889D0A8958BD00CE008B940
:1009400000000000419A000000000000419881D0A2
:10095000A8950CE008B900000000419A00000000D2
:100960000000419872D000E20093080000000000EF
:10097000419A000000000000419867D008E233D09F
:1009800064D00CE030D061D0A89501E02CD061D0CB
:1009900060D05FD006E027D00895B1E0A0E300E288
:1009A00010E20D931A95E9F708950091010100FFF7
:1009B00008950E7F00930101B1E0A0E3A30FB21DE3
:1009C000303021F400E000680ED03FD0303121F407
:1009D00000E4006808D039D00C911DD03395303236
:1009E00009F433270895102F169516951C7318B91E
:1009F000000000000000419A000000004198000F34
:100A0000000F0C7308B9000000000000419A0000BC
:100A1000000041980895102F169516951C731160CB
:100A200018B9000000000000419A00000000419841
:100A3000000F000F0C73016008B9000000000000F7
:100A4000419A000000004198089502E80A95F1F7E4
:100A50000895002711270A95F1F71A95E1F70895EF
:100A6000102F107F1295E12E10E3E10E1AE3E1162C
:100A700010F017E0E10E102F1F70D12E10E3D10EF1
:100A80001AE3D11610F017E0D10E0895DD24EE24FC
:100A9000FF24043618F00456F394FBCF0A3018F004
:100AA0000A50E394FBCFD02E00E3F00EE00ED00E00
:020AB0000895A7
:00000001FF
